:105F2C0001130000F00101010200000301FA04005A
:105F3C00FA0500030A0A5A0B001E0C00FA0D0003A6
:105F4C000E00030F0164100096120132130AFA14AA
:105F5C00010215000017010A1801FA1905321A017D
:105F6C000A1B01FA1C05321FFFFF20FFFF23011E35
:105F7C002400642A00FA2B00FA2C50782D003C2EB9
:105F8C0000462F001E3000643250783432FA35014E
:105F9C0064360164370150380A643C00643E003CAE
:105FAC003F000040FFFF411450420A5A430AC844C4
:105FBC0005324500B44600FA47FFFF4801024C0089
:105FCC00FA4EFFFF50030C510596520A32530B4602
:105FDC00540A96560101570546580002590A465A6A
:105FEC0032FA5B010A5C0A325E000A5F00FE61FF56
:105FFC00FF64FFFF6600026701016A0A3C6B000048
:10600C006C32967300007400007801327901327E94
:10601C00FFFF81FFFF84FFFF8500AF860001870033
:10602C00FA89010A8A00009900009D0A969E0001D7
:10603C009FFFFFFAFAFA0065006F00790083008D6C
:10604C00009700A100AC00B600C000CA00D400DE6E
:10605C0000E800F2005B0063006A0072007A0082C4
:10606C0000890091009900A100A800B000B800BF01
:10607C0000C700CF00D600DF00E600EE00F60040BF
:10608C000046004C00520059005F0065006B007127
:10609C000077007D00830089008F0095009C00A292
:1060AC0000A800AE00B400BA00C000C600CC00D2FC
:0A60BC0000D900DF00E500EB00F161
:1035E7009007A9E0FEA3E0FF905F2E1261FFE4932E
:1035F700F599905F2CE493FC740193FDEFB50507F3
:10360700EEB504037579009007A91261E622AE377B
:10361700AF3874B48E048F05FF1261C88C398D3AA8
:10362700AE37AF3874B48E048F05FF1261F38C3751
:103637008D38E5384537601374B4C39538FFE49582
:1036470037FE8E378F38783912622CE552A839B891
:103657000015D3953A4010E552C3953AFFE49539E2
:10366700FE8E398F3A8010E5522402C3953AFFE463
:103677009539FE8E398F3A22900079E0B40104C261
:10368700108002D21090007AE0B40104C2118002C7
:10369700D2119000B7E075F0C3A4FFAEF0740A8EA4
:1036A700048F05FF1261C890079FECF0A3EDF0743B
:1036B700038C068D071261D8740112003990079D9B
:1036C700EEF0A3EFF074031261D874011200399081
:1036D700000DEEF0A3EFF09000C3E060139000C37D
:1036E700E0F5F0741684FD7C00ED9007ADF08006E0
:1036F70074649007ADF09000B9E090005AF0900123
:1037070003E0900044F0900092E0900046F09000B3
:10371700BBE0900047F0900067E0900048F0900011
:10372700EDE090004DF09000B5E0B40A06740F90FC
:103737000032F09000B5E0B40A0674089000B5F0C6
:103747009000B5E0B40C067535287536179000B5AE
:10375700E0B4080675353C7536E19000B5E0B4066F
:103767000675355075362E9000B5E0B405067535EB
:10377700627536A09000B5E0B404067535767536E7
:10378700CA9000B5E0B403067535A075365C9000A5
:10379700A0E0B40105753D00801F7E017F00900009
:1037A70075E01261D89000B8E08E048F05FF1261B2
:1037B700C8740AFF1261C88D3D9000C1E075F0C35F
:1037C700A4FFAEF0740A8E048F05FF1261C890073C
:1037D700A3ECF0A3EDF09000B5E0B40C0375500630
:1037E7009000B5E0B408037550099000B5E0B40641
:1037F7000375500C9000B5E0B4050375500C9000AC
:10380700B5E0B404037550129000B5E0B403037536
:1038170050189000B5E0B40C09900065E0D3943BD4
:1038270050028006743B900065F09000B5E0B40844
:1038370009900065E0D394595002800674599000AE
:1038470065F09000B5E0B40609900065E0D3947781
:10385700500280067477900065F09000B5E0B405DB
:1038670009900065E0D3948F50028006748F900012
:1038770065F09000B5E0B40409900065E0D394B317
:103887005002800674B3900065F09000B5E0B40371
:1038970009900065E0D394EF5002800674EF900022
:1038A70065F0AE35AF3674021261D890001FEEF0A6
:1038B700A3EFF09000B5E0C39405500A90001F7481
:1038C700FDF0A374E8F090005DE4F0900065E090EF
:1038D700005EF074019000ADF0900035E0D39403E2
:1038E700405A9000B5E0B4060890005D7401F0807E
:1038F7003F9000B5E0B40508740390005DF0803098
:103907009000B5E0B40812740290005DF090006575
:10391700E0245A90005EF080179000B5E0B40C10D8
:10392700740390005DF0900065E0243C90005EF029
:1039370074029000ADF074009000CBF074E3900037
:1039470059F09000A2E0B40B0874E3900059F0809E
:103957005A9000A2E0B419129000B8E090602D12BE
:10396700008CE493900059F080419000A2E0B41ECF
:10397700129000B8E090604B12008CE493900059CD
:10398700F080289000A2E0B428129000B8E0906080
:103997007512008CE493900059F0800F9000A2E01C
:1039A700B44608900099E0900059F0900035E0C3C4
:1039B7009405500D9000BDE0B4020674019000BD5F
:1039C700F0900064E0FE9000B5E0B5063F90005F20
:1039D700E0FE90009FE0B50633900061E0FE9000A6
:1039E700BDE0B50627900060E0FE9000CBE0B5068D
:1039F7001B900063E0FE900072E0B5060F90006236
:103A0700E0FE9000ADE06E7003023B35900035E0BC
:103A1700C39404500874029000EEF080289000359B
:103A2700E0C39404500874069000EEF080179000ED
:103A37005DE0C394035008740A9000EEF0800674AA
:103A4700069000EEF0900035E0D394044009900012
:103A5700BDE0D394015002800874179000F0F08005
:103A67000674009000F0F090009FE06008741A90D0
:103A77000086F0800C7400900086F0740090008738
:103A8700F090009FE0B402087419900087F0800658
:103A97007400900087F09000CBE0701474069006D5
:103AA700C7F074059006CBF074049006CFF080241D
:103AB70074009006C7F074009006C8F07400900672
:103AC700CBF074009006CCF074009006CFF0740031
:103AD7009006D0F0D22690009FE090005FF0900013
:103AE700CBE0900060F09000BDE0900061F09000A6
:103AF700ADE0900062F0900072E0900063F09000FB
:103B0700B5E0900064F0900072E0900045F09000FE
:103B1700ADE0900049F09000CBE090004AF09000B3
:103B27009FE090004BF09000BDE090004CF09000BB
:103B3700D5E0B4011790001B740FF0A374FFF09049
:103B4700001DE4F0A3F074029000D5F09000D5E0DA
:103B5700B4034190001DE0FEA3E0FF90001BE0FCD2
:103B6700A3E0FD12622474101261D87408120039A0
:103B7700EF900056F0EF700674FF900056F0740057
:103B87009000D5F090001CE0900057F090001BE0EB
:103B9700900058F075280122C293C294C291C29234
:103BA700C287C290E5B554EFF5B5E5B554DFF5B575
:103BB700C296C295C2A0C297C2A2C2A1E5B554BF20
:103BC700F5B5E5B5547FF5B5E5B554FBF5B5C212C6
:103BD700753B469000AFE07005754A028003754A51
:103BE70003752C00752B0090000874FFF0A374DC9C
:103BF700F0C218C21A74C8900027F074C890002940
:103C0700F0752A00752900C20D757200E54CB409DC
:103C170003754C00754000900011E4F0A3F0754D5A
:103C270010C215C216C21790079FE0FEA3E0FF74EB
:103C3700031261D8740112003990079DEEF0A3EFCB
:103C4700F0C202C221752E00752D00C22775300003
:103C5700752F00900071E075F032A4FDACF0900074
:103C670019ECF0A3EDF0C23775510090002174FFF5
:103C7700F0A374DCF090002574FFF0A374DCF090DF
:103C87000023E4F0A3F02275A71085F95285FA53B3
:103C97007E017F00E5531261D8E5522FFF50010ED8
:103CA7008E378F38AC39AD3AEF2DFDEE3CFC8C39B1
:103CB7008D3AD293D294D291D292D287D290E53ACA
:103CC700F5FBE539F5FCE53AF5E9E539F5EAE53AD5
:103CD700F5EBE539F5ECE53AF5EDE539F5EEE53ADD
:103CE700F5FDE539F5FEE53AF5CEE539F5CF75A7EA
:103CF700002285F95285FA537E017F00E553126150
:103D0700D8E5522FFF50010E8E378F387E017F7610
:103D17009000EAE01261D8AC37AD38ED2FFFEC3EEA
:103D2700FE8E398F3AE53AF5E9E539F5EA90005A1A
:103D3700E4F07412900032F022A215B3B35006E5F6
:103D47003B64016002807FA201B35006A200B3B3B7
:103D57004002806E75A71085F95285FA537E017F60
:103D670000E5531261D8E5522FFF50010E8E378FB1
:103D77003890000FE0FCA3E0FDEF2DFDEE3CFC8C3E
:103D8700398D3AE53AF5FBE539F5FCE53AF5EBE52A
:103D970039F5ECD293A202B34002D2919000CBE066
:103DA700B4021CAE37AF38AC58AD59EF2DFDEE3C21
:103DB700FC8C398D3AE53AF5EBE539F5ECD291759E
:103DC700A700C215D216A216B3B35006E53B64028C
:103DD7006002807FA201B35006A200B3B340028005
:103DE7006E75A71085F95285FA537E017F00E5535A
:103DF7001261D8E5522FFF50010E8E378F38900091
:103E07000FE0FCA3E0FDEF2DFDEE3CFC8C398D3A75
:103E1700E53AF5E9E539F5EAE53AF5EDE539F5EE9F
:103E2700D294A202B34002D2929000CBE0B4021C1B
:103E3700AE37AF38AC58AD59EF2DFDEE3CFC8C39A1
:103E47008D3AE53AF5EDE539F5EED29275A700D250
:103E570015C21622A215B3B35006E53B64016002F2
:103E6700804FA201B35006A200B3B34002803C7555
:103E7700A71085F95285FA537E017F00E553126139
:103E8700D8E5522FFF50010E8E378F3890000FE084
:103E9700FCA3E0FDEF2DFDEE3CFC8C398D3AE53AB5
:103EA700F5FBE539F5FCD29375A700C215D216D2FA
:103EB70017A216B3B35006E53B64026002804FA217
:103EC70001B35006A200B3B34002803C75A710852A
:103ED700F95285FA537E017F00E5531261D8E55206
:103EE7002FFF50010E8E378F3890000FE0FCA3E0B4
:103EF700FDEF2DFDEE3CFC8C398D3AE53AF5E9E511
:103F070039F5EAD29475A700D215C216D217A217AF
:103F1700B3B35006E53B64036002804FA201B35080
:103F270006A200B3B34002803C75A71085F95285FD
:103F3700FA537E017F00E5531261D8E5522FFF50F7
:103F4700010E8E378F3890000FE0FCA3E0FDEF2DB8
:103F5700FDEE3CFC8C398D3AE53AF5EBE539F5ECAD
:103F6700D29175A700D215D216C21722A215B3B3E4
:103F77005006E53B64016002804DA201B35006A2E2
:103F870000B3B34002803C75A71085F95285FA53F8
:103F97007E017F00E5531261D8E5522FFF50010ED5
:103FA7008E378F3890000FE0FCA3E0FDEF2DFDEE7C
:103FB7003CFC8C398D3AE53AF5FBE539F5FCD293B3
:103FC70075A700C215D216A216B3B35006E53B6417
:103FD700026002804DA201B35006A200B3B34002B3
:103FE700803C75A71085F95285FA537E017F00E55D
:103FF700531261D8E5522FFF50010E8E378F38903C
:10400700000FE0FCA3E0FDEF2DFDEE3CFC8C398DAD
:104017003AE53AF5E9E539F5EAD29475A700D215FC
:10402700C216A215B3B35006E53B64036002804D88
:10403700A201B35006A200B3B34002803C75A7109B
:1040470085F95285FA537E017F00E5531261D8E561
:10405700522FFF50010E8E378F3890000FE0FCA3D0
:10406700E0FDEF2DFDEE3CFC8C398D3AE53AF5EBA2
:10407700E539F5ECD29175A700C215D216A216B391
:10408700B35006E53B64046002804DA201B35006BD
:10409700A200B3B34002803C75A71085F95285FA98
:1040A700537E017F00E5531261D8E5522FFF50017F
:1040B7000E8E378F3890000FE0FCA3E0FDEF2DFD4B
:1040C700EE3CFC8C398D3AE53AF5EDE539F5EED263
:1040D7009275A700D215C21622A215B3B35006E5F2
:1040E7003B64016002804FA201B35006A200B3B344
:1040F7004002803C75A71085F95285FA537E017FEF
:1041070000E5531261D8E5522FFF50010E8E378F0D
:104117003890000FE0FCA3E0FDEF2DFDEE3CFC8C9A
:10412700398D3AE53AF5FBE539F5FCD29375A700E9
:10413700C215D216D217A216B3B35006E53B6402D6
:104147006002804FA201B35006A200B3B3400280C1
:104157003C75A71085F95285FA537E017F00E55318
:104167001261D8E5522FFF50010E8E378F3890001D
:104177000FE0FCA3E0FDEF2DFDEE3CFC8C398D3A02
:10418700E53AF5E9E539F5EAD29475A700D215C203
:1041970016D217A217B3B35006E53B64036002803B
:1041A7004FA201B35006A200B3B34002803C75A7EB
:1041B7001085F95285FA537E017F00E5531261D8C5
:1041C700E5522FFF50010E8E378F3890000FE0FC1D
:1041D700A3E0FDEF2DFDEE3CFC8C398D3AE53AF579
:1041E700EBE539F5ECD29175A700D215D216C217B7
:1041F700A215B3B35006E53B64046002804FA201E9
:10420700B35006A200B3B34002803C75A71085F9EE
:104217005285FA537E017F00E5531261D8E5522F8C
:10422700FF50010E8E378F3890000FE0FCA3E0FDA2
:10423700EF2DFDEE3CFC8C398D3AE53AF5EDE5398D
:10424700F5EED29275A700C215D216D217A216B3F1
:10425700B35006E53B64056002804FA201B35006E8
:10426700A200B3B34002803C75A71085F95285FAC6
:10427700537E017F00E5531261D8E5522FFF5001AD
:104287000E8E378F3890000FE0FCA3E0FDEF2DFD79
:10429700EE3CFC8C398D3AE53AF5FDE539F5FED271
:1042A7008775A700D215C216D217A217B3B3500647
:1042B700E53B64066002804FA201B35006A200B33B
:1042C700B34002803C75A71085F95285FA537E01E9
:1042D7007F00E5531261D8E5522FFF50010E8E374C
:1042E7008F3890000FE0FCA3E0FDEF2DFDEE3CFCC6
:1042F7008C398D3AE53AF5CEE539F5CFD29075A7E9
:1043070000D215D216C21722054122A2D8B3400205
:10431700D221A2D8B34002C296A2D9B340089000D6
:10432700B9E090005AF075D8402285A74F75A710BD
:10433700A2D8B34002C293A2D9B34002C294A2DA70
:10434700B34002C291A2DBB34002C292A2DCB340E7
:1043570002C287A2DDB34002C29075D840854FA73D
:1043670022900047E4936406600280FE74C89007B9
:10437700A5F8E4F0E8A3F075B50075840175A7000A
:1043870075FFA090002FE4F075C91075A70F75A1F0
:10439700C775A70075D90075CE0C75A70F75F1FE07
:1043A70075F2FF75F30775F47875A4BA75A5FF75EF
:1043B700A60775AE0075AFFF75D48175D5FF75D6A5
:1043C700FF75D7FF75A70075A20175A14775F80995
:1043D70075D80075D90475DA0975D84075A71075B1
:1043E700D80075D90475DA0975DB0975DC0975DD3F
:1043F7000975DE0975DF0975D84075A70075E608E8
:1044070075E71075BC0175BE0475BD6C75BE077583
:10441700BDA075BE0875BD0175BC0075BB1875BC20
:104427002075BA0875E88075D11375A70F75E10572
:1044370075E20075C740123B9F75970075978074AA
:104447000A1261B87597C0E5975420700280F87515
:104457008F0275A700D2AF75980075A90C75A70FC5
:1044670075AB4375ADFB75AC1E75A71075C918758F
:10447700CA0075CB0075C80475A700758912758EBB
:1044870004758C00758A00C2A9D28C758D00758B56
:1044970000D2ABD28E75EF0675D944C29974C8F5B0
:1044A700097508001200E375B5001204E374639000
:1044B70007A5F8E4F0E8A3F012036F74C89007A506
:1044C700F8E4F0E8A3F07464F5097508001200E356
:1044D700900045E0900072F0C21E900072E0D39405
:1044E7000340067400900072F0900072E0905B4702
:1044F700F82828738028A2B44002D21E802075A70E
:104507000F75F30F75A700A2A34002D21E800F7587
:0E451700A70F75F31775A700A2A44002D21ECD
:0C5B47000244FB0244FD02450502451625
:10452500A21EB34066755208E552D3940E5020E59D
:10453500529007A5F8E4F0E8A3F012023E7464F582
:10454500097508001200E37852740126F650D974F3
:10455500029000AEF0900072E0D394034006740020
:10456500900072F0900072E0905B53F828287380F9
:104575001674009000D8F0800E74009000BDF08095
:074585000674009000CAF06B
:0C5B530002457402457602457E0245863C
:10458C00D21D8064755201E552D394075020E55238
:10459C009007A5F8E4F0E8A3F012023E7464F50964
:1045AC007508001200E37852740126F650D9740194
:1045BC009000AEF0900072E0D3940340067400902B
:1045CC000072F0900072E0905B5FF8282873801600
:1045DC0074009000D8F0800E74009000BDF080063E
:0645EC0074009000CAF00B
:0C5B5F000245DA0245DC0245E40245EC98
:1045F200C21D900044E0900103F0900045E090005D
:1046020072F0900046E0900092F0900047E0900037
:10461200BBF0900048E0900067F0900049E0900005
:10462200ADF090004AE09000CBF090004BE090009B
:104632009FF090004CE09000BDF090004DE09000A3
:10464200EDF09000B8E07006740A9000B8F09000A7
:1046520099E0700674E3900099F090009FE0049056
:10466200005FF012367FE5B54401F5B5740690009F
:1046720033F07401900034F07403900036F0740546
:10468200900037F07401900038F07403900039F014
:10469200900035E0B404067404900039F0900035BF
:1046A200E0B405067405900039F0740090003AF009
:1046B200740090003FF07400900040F0740190008C
:1046C20041F07400900042F074FF900043F0745384
:1046D20090013CF0747490013DF0746190013EF0E1
:1046E200746E90013FF07464900140F07461900127
:1046F20041F07472900142F07464900143F07420AE
:10470200900144F07450900145F07475900146F0A8
:10471200746C900147F07473900148F074659001D5
:1047220049F0747390014AF09000D4E0900056F082
:1047320090008BE0900057F090008CE0900058F0D1
:10474200A2B6B3920EA2B3B3920FA2A4B39223A2C3
:10475200B4B39224A2A3B39225900052E4F0754C14
:1047620000743A900765F074FD900766F09000536C
:10477200E4F090079FE0FEA3E0FF74031261D87497
:104782000112003990079DEEF0A3EFF0754B0190F6
:104792000032E4F0C222754000C213D214C2027584
:1047A2004E00C229D203C22AD204C22BD205C22C85
:1047B200D206C22DD207C22ED208C22FD209C230CF
:1047C200D20AC231D20BC232D20CC21FC220C226BE
:1047D20012009E753C00754800753E0075423275A8
:1047E200430075440075450075460075470090000A
:1047F20011E4F0A3F0754900D2B2D2A4D2B0D2B182
:10480200D2A3D2A7D2A6D2A5D2B7900071E0D394F8
:10481200FA400674FA900071F07E017F0090005811
:10482200E01261D8900057E02FFF50010E90001B5C
:10483200EEF0A3EFF0EFD394FFEE940F4007900059
:104842001BE4F0A3F0900056E0700674FF9000564F
:10485200F07400900098F09000AEE0D3940240060D
:1048620074019000AEF09000AFE07005754A0280CE
:1048720003754A039000B0E0D3940140067400909F
:1048820000B0F09000B6E0C3940A5006740A90009B
:10489200B6F09000C0E0700674019000C0F0900085
:1048A200C0E0B4FF0674FE9000C0F09000C7E0D3F1
:1048B20094FE400674FE9000C7F09000EDE0D394A1
:1048C20002400674019000EDF0900103E0D39401E0
:1048D20040067401900103F074019000CDF0740160
:1048E2009000CEF074009000D5F074009000F5F0C6
:1048F20074299006ABF0742A9006AFF074169006F5
:10490200B3F074079006B7F074089006BBF0741BFE
:104912009006BFF0741C9006C3F0D29C9000A0E0F9
:10492200D39404400674049000A0F09000D2E0D327
:104932009404400674049000D2F0E54DD3941040E4
:1049420003754D109006ACE0D3940C4006740090B1
:1049520006ACF09006B0E0D3940C400674009006CA
:10496200B0F09006B4E0D3940C400674009006B404
:10497200F09006B8E0D3940C400674009006B8F0AC
:104982009006BCE0D3940C400674009006BCF090F4
:1049920006C0E0D3940C400674009006C0F0900666
:1049A200C4E0D3940C400674009006C4F09006C88C
:1049B200E0D3940C400674009006C8F09006CCE058
:1049C200D3940C400674009006CCF09006D0E0D34D
:1049D200940C400674009006D0F0D2EC75CF01A280
:1049E20098B34005C298120616E5796006A299B3FB
:1049F200B340028005C299120AB4E57A64016005E7
:104A0200E57AB4040280D5C28E7E107F00E54112A1
:104A120061D8E58D75F010A4FDACF0EF2DFDEE3CF4
:104A2200FCE58B75F01084FF7E00ED2FFFEC3EFE5F
:104A32008E2B8F2CD28E900092E060569000131233
:104A420061E6900013E0FCA3E0FD900015E0FAA3FC
:104A5200E0FBEDB5033CECB50238B21CA20DB3404D
:104A620013A21CB34008E5B54404F5B58006E5B5CC
:104A720054FBF5B5900015E0FEA3E0FF900017E0AF
:104A8200FCA3E0FDEF2DFDEE3CFC900015ECF0A345
:104A9200EDF090009FE0600990009FE0C394034016
:104AA20002806F1229C0A20DB35009900052E0C3D8
:104AB200940740028006900089E0F571E57175F077
:104AC20005A4FFAEF09007A7EEF0A3EFF0900076FA
:104AD200E0C3953E4007E53CC3953D50079007A7CC
:104AE200E4F0A3F0AE5AAF5B9007A7E0FCA3E0FDB1
:104AF200EFD39DEE9C4004C2A1800B900052E0C314
:104B0200940B5002D2A190009FE0B40205A2A1B37F
:104B120092A290009FE0B4031C122ADBAE5AAF5B54
:104B22009007A7E0FCA3E0FDEFD39DEE9C4004D2EA
:104B3200A18002C2A1A2B6300E01B35003025023DB
:104B4200A2B6300E01B35003025023A2B6301001B8
:104B5200B35003024E79754B00053BE54AB403544A
:104B6200AE2BAF2C7401120039900008E0FCA3E0D8
:104B7200FD74038F02FF1261C8EDC39AEC9E4022BE
:104B8200AE2BAF2C74038E048F05FF1261C8900008
:104B920008E0FEA3E0FF7401120039EFD39DEE9C02
:104BA2004005754A01800BA227B34006900032747B
:104BB20001F0D227E54AB40203754A01AE2BAF2CAD
:104BC2007401120039900008E0FCA3E0FD74038F29
:104BD20002FF1261C8EAC39DEE9C4022AE2BAF2CAD
:104BE20074038E048F05FF1261C8900008E0FEA3D3
:104BF200E0FF7401120039EDD39FEC9E400674026F
:104C0200900032F0900008E52BF0A3E52CF0AE2BDB
:104C1200AF2CE5508E048F05FF1261C88C2D8D2EAE
:104C2200AE2BAF2C74011200398E338F34AC2FAD02
:104C320030AA2BAB2CED2BFBEC3AFA8A2F8B30AC43
:104C42002BAD2CEDD39BEC9A401190000BE0F9A315
:104C5200E0FEEEC394E8E994034002800690000B64
:104C62001261E6900092E06043900013E0FEA3E040
:104C7200FF900092E08E048F05FF1261C874018CD0
:104C8200068D07120039900017EEF0A3EFF09000A6
:104C920017E0F8A3E0900015C8F0A3C8F090001345
:104CA200E4F0A3F0C21CE5B554FBF5B5C28E758DD8
:104CB20000758B00754100752C01752B00D28E900A
:104CC2000008E0FEA3E0FFEF4E601074011200390D
:104CD200AC35AD361260C68E298F2AAE29AF2A7442
:104CE20028BE00039F5010E5402FFF50010E7401B3
:104CF2001200398E298F2A852A409000B6E0A82911
:104D0200B8000DD3952A4008E52A900031F08009B9
:104D12009000B6E014900031F0E54A6006752A0072
:104D220075290012202BA212B35003024E319000BB
:104D32005DE0905B6BF8282873E53BD39402400357
:104D4200753B018037E53BD394034003753B0180FB
:104D52002BE53BD394044003753B01801F9000B5C3
:104D6200E0B40507E53BD3940550028005753B018D
:0C4D7200800AE53BD394064003753B012A
:0C5B6B00024D3B024D47024D53024D5FBE
:104D7E00A213B35006A212B3B34003024E319000F9
:104D8E006BE0B401739000EDE0B40214120C559078
:104D9E00005BE075F0BEA4FFAEF08E398F3A805600
:104DAE00E54475F00A84FF7E009005651261FFE010
:104DBE00F538753700AE37AF38900090E01261D8F5
:104DCE0074648E048F05FF1261C88C398D3AE53AF2
:104DDE0090000AF0AE37AF38900069E01261D874D7
:104DEE00648E048F05FF1261C874BE8C068D071287
:104DFE0061D88E398F3A8017900069E075F0BEA4A5
:104E0E00FFAEF08E398F3A900090E090000AF0E5F8
:104E1E003EC394CC5006900069E070028003123CB1
:104E2E008ED213E54AB40103754D01E54A703790F1
:104E3E0000B2E0D39401400D90005AE0A829B800CA
:104E4E0006952A4002801C9000B2E0B40305754D11
:104E5E00038002C20090005AE0600674099000328E
:104E6E00F08003754D01A210B3920EA210B330B6AE
:104E7E0001B35003025023754B01E5B54401F5B55E
:104E8E007407900052F0A210920EE53BD394474067
:104E9E0002D212E54CB40903754C009000BAE0B48E
:104EAE000107E547C3941440028009123B9F741317
:104EBE00900032F0A229300301B35017A229B3405B
:104ECE0008E5B54408F5B58006E5B554F7F5B5A285
:104EDE00299203A22A300401B35017A22AB3400824
:104EEE00E5B54402F5B58006E5B554FDF5B5A22A43
:104EFE009204A22B300501B3500FA22BB34004D263
:104F0E00958002C295A22B9205A22C300601B350B9
:104F1E0017A22CB34008E5B54410F5B58006E5B5EB
:104F2E0054EFF5B5A22C9206A22D300701B35017FF
:104F3E00A22DB34008E5B54420F5B58006E5B5547D
:104F4E00DFF5B5A22D9207A22E300801B35017A29D
:104F5E002EB34008E5B54440F5B58006E5B554BF1F
:104F6E00F5B5A22E9208A22F300901B35017A22F29
:104F7E00B34008E5B54480F5B58006E5B5547FF538
:104F8E00B5A22F9209A230300A01B3500FA230B34E
:104F9E004004D2908002C290A230920AA231300B0D
:104FAE0001B3500FA231B34004D2878002C287A250
:104FBE0031920BA232300C01B3500FA232B3400427
:104FCE00D2928002C292A232920CE547C394415013
:104FDE0009740E900032F0123B9F900039E0FE9063
:104FEE000035E004C39E4009900035E0D39406409E
:104FFE000974FB900032F0123B9F90003EE060156A
:10500E0090003EE0FE900038E06E600974FE900065
:10501E0032F0123B9F90005DE0905B77F82828738A
:10502E00123D40800D123E5B8008123F73800312CA
:02503E0040E050
:0C5B770002502E02503302503802503D04
:10504000E54D905B83F82828730257169000D2E054
:065B830002504902504CE3
:10505000905BB6F8282873121B078012121B07807A
:0E5060000D121B918008121C3D8003121C3D96
:0F5BB60002505702505C02506102506602506B61
:10506E00754D02025716121D69121E80A237B340EB
:10507E000C900094E0F5497410900032F085496070
:10508E00900008E0FEA3E0FF90000DE0FCA3E0FD21
:10509E00EDD39FEC9E401974021261D874038E04F6
:1050AE008F05FF1261C8900000ECF0A3EDF0800FA9
:1050BE0090079DE0F8A3E0900000C8F0A3C8F0753B
:1050CE004D03A2384003754D0A0257169006ACE008
:1050DE0060031221149000EBE0B401149000ECE098
:1050EE00A829B80004952A5007E53CC3953D400217
:1050FE0080030251849000A0E0D39402403F9000C0
:10510E0074E02403A829B80004952A50099000766B
:10511E00E0D3953E50028008D2017408900032F020
:10512E00900074E0A829B80005D3952A500B900082
:10513E0076E02403C3953E5002C20180399000747C
:10514E00E02403A829B80004952A5007E53CC3952E
:10515E003D40028008D2017408900032F090007435
:10516E00E0A829B80005D3952A5009E53D240FC3C0
:10517E00953C5002C2019000BAE07007E547C39417
:10518E001440028002D201A2014005754D04800A2E
:10519E00754D10900011E4F0A3F0A20DB3405DE543
:1051AE004475F00A84FF7E009005651261FFE0C32E
:1051BE009469501F12206090079DE0FEA3E0FF74DB
:1051CE00031261D8740112003990000DEEF0A3EFB6
:1051DE00F0802990079FE0F8A3E090079DC8F0A308
:1051EE00C8F090079DE0FEA3E0FF74031261D8742F
:1051FE000112003990000DEEF0A3EFF00257169059
:03520E0000A0E01D
:095B89000250740250DA02520DC0
:10521100905BC5F8282873120D3F8012120D3F8054
:0E5221000D120EED8008120F9F8003120F9FDA
:0F5BC50002521802521D02522202522702522C83
:10522F009006B0E060031221F0754D05025716127B
:10523F0010AB754D069006B4E060031222E09006A5
:10524F00B8E060031223BC02571690000AE0600614
:10525F00A20DB3B34002801D90000AE02555FFAEAA
:10526F005450010E8E548F55E53BD3940150069048
:10527F00000AE014F01212F1754D079006BCE060C1
:10528F00031224989006C0E060031225740257168B
:10529F009000EDE0B40203120CCD12154E754D08BF
:1052AF009006C4E060031226509006C8E060031217
:1052BF00272C02571612190AA215B35005A216B3BE
:1052CF0040028006D215D216D217754D109006CC1B
:1052DF00E060031228089006D0E060031228E40271
:1052EF0057160257169000B5E0B40502800302541A
:1052FF007790005EE0D3956050030253E1AE29AF83
:10530F002A740ABE00039F501EAE2DAF2E90005E72
:10531F00E0C395601261D8740C8E048F05FF126183
:10532F00C88C318D328020AE2DAF2E740C8E048F31
:10533F0005FF1261C890005EE0C395608C068D0773
:10534F001261D88E318F32900000E0FEA3E0FFACE7
:10535F0031AD32EDD39FEC9E40288F028E038C0629
:10536F008D078B048A05126224900023EEF0A3EFC1
:10537F00F0E551B40207900023E4F0A3F07551005B
:10538F00804EE5517003755101900008E0FEA3E0D7
:10539F00FFAC31AD32EF2DFDEE3CFC900000E0FA9A
:1053AF00A3E0FBEDD39BEC9A401FAC31AD32EF2D58
:1053BF00FDEE3CFC8C068D078A048B05126224904F
:1053CF000023EEF0A3EFF08007900023E4F0A3F0AA
:1053DF008074AE2DAF2E90005EE0F4042560126154
:1053EF00D8740C8E048F05FF1261C88C318D3290EA
:1053FF000000E0FEA3E0FFED2FFFEC3EFE90000863
:10540F00E0FAA3E0FBEBD39FEA9E401C8A068B07D2
:10541F00126224900000E0FCA3E0FD1262249000D1
:10542F0023EEF0A3EFF0801E900023E4F0A3F090A2
:10543F000008E0FEA3E0FFAC31AD32126224900011
:10544F0000EEF0A3EFF0900000E0FEA3E0FF741376
:10545F001261D874148E048F05FF1261C89000007A
:10546F00ECF0A3EDF002562690005EE0D39560506D
:10547F0003025559AE29AF2A740ABE00039F501E6E
:10548F00AE2DAF2E90005EE0C395601261D8740A06
:10549F008E048F05FF1261C88C318D328020AE2DA6
:1054AF00AF2E740A8E048F05FF1261C890005EE064
:1054BF00C395608C068D071261D88E318F329000A4
:1054CF0000E0FEA3E0FFAC31AD32EDD39FEC9E4088
:1054DF00288F028E038C068D078B048A0512622497
:1054EF00900023EEF0A3EFF0E551B40207900023F4
:1054FF00E4F0A3F0755100804EE551700375510132
:10550F00900008E0FEA3E0FFAC31AD32EF2DFDEED1
:10551F003CFC900000E0FAA3E0FBEDD39BEC9A403B
:10552F001FAC31AD32EF2DFDEE3CFC8C068D078AA2
:10553F00048B05126224900023EEF0A3EFF0800796
:10554F00900023E4F0A3F0025607AE29AF2A740AA5
:10555F00BE00039F501FAE2DAF2E90005EE0F404EF
:10556F0025601261D8740A8E048F05FF1261C88CF2
:10557F00318D328021AE2DAF2E740A8E048F05FF30
:10558F001261C890005EE0F40425608C068D07124E
:10559F0061D88E318F32AE31AF32900000E0FCA374
:1055AF00E0FDEF2DFDEE3CFC900008E0FAA3E0FBE0
:1055BF00EBD39DEA9C40238F048E058A068B07CD83
:1055CF00CCCD126224900000E0FCA3E0FD12622417
:1055DF00900023EEF0A3EFF0801E900023E4F0A3E1
:1055EF00F0900008E0FEA3E0FFAC31AD3212622470
:1055FF00900000EEF0A3EFF0900000E0FEA3E0FFBC
:10560F0074131261D874148E048F05FF1261C89041
:10561F000000ECF0A3EDF0E551B40149755102E53E
:10562F004A703685F95285FA537E017F00E5531291
:10563F0061D8E5522FFF50010E8E378F3890000042
:10564F00E0FCA3E0FDEF2DFDEE3CFC8C398D3AE53F
:10565F003AF5FBE539F5FCD29690002174FFF0A3E3
:10566F0074DCF0807C900021E0FEA3E0FFEFB4DC5F
:10567F002CEEB4FF28900025E0FCA3E0FDEDB4DC98
:10568F001AECB4FF16900023E0F8A3E0900021C8B5
:10569F00F0A3C8F0900023E4F0A3F08044E54A7033
:1056AF003685F95285FA537E017F00E5531261D892
:1056BF00E5522FFF50010E8E378F38900000E0FC1F
:1056CF00A3E0FDEF2DFDEE3CFC8C398D3AE53AF56C
:1056DF00FBE539F5FCD29690002174FFF0A374DC42
:1056EF00F0E54AB40112754A00754D10900021740F
:1056FF00FFF0A374DCF08003754D03800A800880EF
:07570F000680048002800007
:105B920002523E02525902529F0252C40252F10272
:105BA20052F402570C02570E0257100257120257B4
:045BB200140257166C
:10571600AE2BAF2C900021E0FCA3E0FDEFD39DEE75
:105726009C4044E54A703685F95285FA537E017FDE
:1057360000E5531261D8E5522FFF50010E8E378FC8
:1057460038900000E0FAA3E0FBEF2BFBEE3AFA8A72
:10575600398B3AE53AF5FBE539F5FCD2969000210E
:1057660074FFF0A374DCF0A221B3402E90002574E0
:10577600FFF0A374DCF0900023E0FEA3E0FFEF4E01
:105786006016900023E0F8A3E0900021C8F0A3C8BB
:10579600F0900023E4F0A3F0C2219000BDE0B40233
:1057A6000280030258BC900054E0D39543506490A5
:1057B6000054E0F4042543FE9000C0E08E00F5F0AE
:1057C600E884FF7E008F52EFC39410500CEF855291
:1057D600F0A4FDACF08D5280037552FF900054E0AA
:1057E600D39552400B900054E0C39552F54E80037A
:1057F600754E009000DBE0D3954E40069000DBE04E
:10580600F54E9000DCE0C3954E50069000DCE0F5C6
:105816004E8071900054E0C39543FE9000C0E08E28
:1058260000F5F0E884FF7E008F52EFC39410500C11
:10583600EF8552F0A4FDACF08D5280037552FF85C2
:105846005238753700900054E02538FFAE375001C6
:105856000E8E378F3874FFBE0009D39F40058538FA
:105866004E8003754EFF9000DBE0D3954E400690C8
:1058760000DBE0F54E9000DCE0C3954E500690004C
:10588600DCE0F54EA20DB3B3500D900055E0FE904E
:1058960000C8E0D39E5002800A7407900032F0C21E
:1058A60097801375A710E5CDC3954E4004C2978027
:1058B60002D29775A700E54CC39409500AA2EDB32E
:1058C6004005C2ED122C7AAE2BAF2C90001FE0FCE7
:1058D600A3E0FDEDC39FEC9E400C900053E0C39403
:1058E6005A4003025B44A212B34009123B9F74065E
:1058F600900032F0A21EB34008E5B54404F5B58029
:1059060006E5B554FBF5B5A214B3500EE53ED394A7
:10591600334007E53EC394CC4002802FE5B54401F1
:10592600F5B57407900052F0900069E075F0BEA4DA
:10593600FFAEF08E398F3A7402BE000AD39F40063E
:10594600753A02753900123C8ED214900053E0D39A
:1059560094014007E53EC3941A40028002C21490A7
:1059660006ACE06003122114A229300301B35017DC
:10597600A229B34008E5B54408F5B58006E5B55457
:10598600F7F5B5A22992039006B0E060031221F064
:10599600A22A300401B35017A22AB34008E5B54441
:1059A60002F5B58006E5B554FDF5B5A22A92049038
:1059B60006B4E060031222E0A22B300501B3500FBB
:1059C600A22BB34004D2958002C295A22B920590D9
:1059D60006B8E060031223BCA22C300601B35017B0
:1059E600A22CB34008E5B54410F5B58006E5B554DC
:1059F600EFF5B5A22C92069006BCE060031224983F
:105A0600A22D300701B35017A22DB34008E5B544C7
:105A160020F5B58006E5B554DFF5B5A22D920790C1
:105A260006C0E06003122574A22E300801B3501799
:105A3600A22EB34008E5B54440F5B58006E5B55459
:105A4600BFF5B5A22E92089006C4E0600312265058
:105A5600A22F300901B35017A22FB34008E5B54471
:105A660080F5B58006E5B5547FF5B5A22F9209906D
:105A760006C8E0600312272CA230300A01B3500F8B
:105A8600A230B34004D2908002C290A230920A9013
:105A960006CCE06003122808A231300B01B3500F88
:105AA600A231B34004D2878002C287A231920B9002
:105AB60006D0E060031228E4A232300C01B3500F86
:105AC600A232B34004D2928002C292A232920C90C9
:105AD6000053E0C3945A5010E54CB40909900053A2
:105AE600E004F0754C00803BE54CB40903754C00AE
:105AF600752C00752B00758D00758B007541009017
:105B06000052E0C3940B5008900052E004F0800667
:105B1600740B900052F0900052E0B40B06E5B554B9
:105B2600FEF5B5900053E0D394014007E547C394D2
:105B36004140028009740E900032F0123B9F0249E8
:015B4600DE80
:105BD4000000010001400160018001A001C001E05A
:105BE40002000300039603B603D603F40400050081
:105BF4000512052405360548055A056C057E0590F1
:105C040005A805C005DE0600061406280646066E2D
:105C140006AE00FF013F015F017F019F01BF01DF6D
:105C240001FF02FF039503B503D503F303FF04FF4C
:105C340005110523053505470559056B057D058FB8
:105C440005A705BF05DD05F1061306270645066D04
:105C540006AD06ED0FAA0FA50F9F0F9A0F940F8D97
:105C64000F870F800F780F710F680F600F570F4E5B
:105C74000F450F3B0F300F250F1A0F0E0F020EF5B5
:105C84000EE80EDB0ECC0EBE0EAE0E9F0E8E0E7DFB
:105C94000E6C0E5A0E470E340E200E0C0DF70DE24C
:105CA4000DCB0DB50D9D0D850D6D0D540D3A0D20CB
:105CB4000D050CE90CCE0CB10C940C760C580C3A76
:105CC4000C1B0BFB0BDB0BBB0B9A0B790B570B352C
:105CD4000B130AF10ACE0AAB0A870A640A400A1CAB
:105CE40009F809D409B0098C09670943091F08FB9D
:105CF40008D608B2088E086A0846082307FF07DC9E
:105D040007B9079607730751072F070D06EC06CA54
:105D140006AA068906690649062A060A05EC05CD7F
:105D240005B0059205750558053C0520050504EAEE
:105D340004CF04B5049C0482046904510439042288
:105D4400040B03F403DE03C803B2039D0389037544
:105D54000361034D033B03280316030402F202E12B
:105D640002D102C002B002A0029102820273026553
:105D740002570249023C022F02220216020901FDC7
:105D840001F201E601DB01D001C601BB01B101A7AB
:105D9400019D0194018B0182017901700168016008
:105DA400015801500148014101390132012B0125FB
:105DB400011E01180111010B010500FF00FA0FA6D5
:105DC4000FA00F990F920F8B0F840F7C0F740F6B22
:105DD4000F620F580F4E0F430F380F2C0F1F0F1267
:105DE4000F050EF70EE80ED80EC80EB70EA50E93CB
:105DF4000E800E6C0E580E420E2C0E150DFD0DE489
:105E04000DCB0DB10D950D790D5D0D3F0D200D01DF
:105E14000CE10CC00C9E0C7C0C590C350C100BEADC
:105E24000BC40B9E0B760B4F0B260AFD0AD40AAA51
:105E34000A800A550A2A09FF09D409A8097C0950CD
:105E4400092508F908CD08A10875084A081E07F3B2
:105E540007C8079D07730749072006F706CE06A65D
:105E6400067E06570630060A05E405BF059B05773E
:105E740005540532051004EF04CE04AE048F0471FA
:105E840004530435041903FD03E203C703AD03946B
:105E9400037B0363034B0334031E030802F302DE94
:105EA40002CA02B602A30291027F026D025C024C96
:105EB400023C022C021D020E020001F201E401D791
:105EC40001CA01BE01B101A6019A018F0185017ABF
:105ED40001700166015D0153014A0141013901313B
:105EE4000129012101190112010B010400FD00F730
:105EF40000F000EA00E400DE00D900D300CE00C9BF
:105F040000C400BF00BA00B500B100AD00A800A4F1
:105F140000A0009C009900950091008E008A0087E3
:085F240000840081007E007B77
:10009E007573009007A9E4F0A3F0755D00755C0020
:1000AE00757900757A00C234D23574FE9007B3F8B4
:1000BE00E4F0E8A3F074FE9007B5F8E4F0E8A3F0DE
:1000CE00745A9007B7F0745A9007B8F0D236C22817
:1000DE00C238C23322750B00750A00AE0AAF0BACE4
:1000EE0008AD09EDC39FEC9E401674FF1261B87502
:1000FE00CF01780B740126F6500418E436F650DB67
:10010E002290002FE0B4AA1C900765E0B43C159035
:10011E0007A5E0FEA3E0FFEF4E6009741EBE0004CB
:10012E00D39F500302023D753A0075390075F809E8
:10013E009007A5E0FEA3E0FF74076F4E6006740EF5
:10014E006F4E7006743A900765F09007A5E0FEA317
:10015E00E0FF7408BE001ED39F401A7E017F0890F8
:10016E0007A5E0FCA3E0FD1DBDFF011C1200038EE0
:10017E00378F38801F9007A5E0FEA3E0FF740812AA
:10018E00621C8F048E057E017F08CDCCCD1200033C
:10019E008E378F38AE39AF3A740CD39F74019E50A0
:1001AE0003020238A2F9B3407EE53A453970037571
:1001BE00A382AE39AF3A74016F4E700375A300AED1
:1001CE0039AF3A74026F4E700D9007A6E075F002CB
:1001DE00A4FDACF08DA3AE39AF3A74036F4E70032D
:1001EE0075A300AE39AF3A7403BE00039F5013AC33
:1001FE0037AD38ED2FFFEC3EFE9000611261FFE04F
:10020E00F5A3AE39AF3AEFB40B09EEB40105741491
:10021E001261B8AE39AF3AEFB40B07EEB401037505
:10022E00F80D783912622C0201A290002FE4F02210
:10023E00753A0075390075F8099007A5E0FEA3E040
:10024E00FF7408BE001ED39F401A7E017F089007E0
:10025E00A5E0FCA3E0FD1DBDFF011C1200038E37BF
:10026E008F38801F9007A5E0FEA3E0FF740812628E
:10027E001C8F048E057E017F08CDCCCD1200038E1F
:10028E00378F38AE39AF3A7411D39F74019E500335
:10029E0002036EA2F9B3500302036BE53A453970BF
:1002AE000375A3D2AE39AF3A74016F4E700375A3C6
:1002BE0000AE39AF3A74026F4E700D9007A6E0751E
:1002CE00F002A4FDACF08DA3AE39AF3A74036F4EBD
:1002DE00700375A300AE39AF3A74046F4E70037598
:1002EE00A300AE39AF3A74056F4E700375A300AE1E
:1002FE0039AF3A74066F4E700375A300AE39AF3A3C
:10030E0074076F4E700375A300AE39AF3A74086F61
:10031E004E700375A300AE39AF3A7408BE00039F4A
:10032E005016AC37AD38ED2FFFEC3EFE90005C1250
:10033E0061FFE5A3F075A300AE39AF3AEFB4100933
:10034E00EEB4010574141261B8AE39AF3AEFB410C1
:10035E0007EEB4010375F80D783912622C02029182
:10036E0022753A0075390075F809AE39AF3A74172F
:10037E00BE0004D39F5003020447A2F9B3500302F8
:10038E000444E53A4539700375A3D2AE39AF3A74D9
:10039E00016F4E700375A300AE39AF3A74026F4E03
:1003AE00700D9007A6E075F002A4FDACF08DA3AE23
:1003BE0039AF3A74036F4E700375A300AE39AF3A7E
:1003CE0074046F4E700375A300AE39AF3A74056FA7
:1003DE004E700375A300AE39AF3A74066F4E7003BC
:1003EE0075A300AE39AF3A74076F4E700375A30054
:1003FE00AE39AF3A74086F4E700375A300AE39AFC5
:10040E003A7408BE00039F500C90003B1261FFE54A
:10041E00A3F075A300AE39AF3A74166F4E70057423
:10042E00141261B8AE39AF3A74166F4E700375F888
:10043E000D783912622C0203782290002FE0B4ABB3
:10044E000280030204E2753A0075390075F809AEB0
:10045E0039AF3A7412BE007CD39F4078A2F9B340F4
:10046E0070E53A4539700375A382AE39AF3A74011F
:10047E006F4E700375A300AE39AF3A74026F4E70B3
:10048E000D9007A6E075F002A4FDACF08DA3AE3979
:10049E00AF3A74036F4E700375A300AE39AF3A7462
:1004AE0003BE00039F50099000401261FFE0F5A3C8
:1004BE00AE39AF3A74116F4E700574141261B8AE46
:1004CE0039AF3A74116F4E700375F80D78391262A8
:1004DE002C02045D229007B0E4F074649007A5F836
:1004EE00E4F0E8A3F012036F74C89007A5F8E4F0E7
:1004FE00E8A3F0900047E0B4371A900044E0900073
:10050E003BF0900045E090003CF0900046E09000FB
:10051E003DF080469007B07401F074659007A5F821
:10052E00E4F0E8A3F012036F74C89007A5F8E4F0A6
:10053E00E8A3F0900047E0B4371A900044E0900032
:10054E003BF0900045E090003CF0900046E09000BB
:10055E003DF0800674029007B0F09007B1E4F0749D
:10056E00669007A5F8E4F0E8A3F012036F74C89044
:10057E0007A5F8E4F0E8A3F0900046E0B437129037
:10058E000044E0900035F0900045E090003EF08091
:10059E00769007B17401F074679007A5F8E4F0E85F
:1005AE00A3F012036F74C89007A5F8E4F0E8A3F067
:1005BE00900046E0B43712900044E0900035F09081
:1005CE000045E090003EF0803E74029007B1F0745A
:1005DE00689007A5F8E4F0E8A3F012036F74C890D2
:1005EE0007A5F8E4F0E8A3F0900046E0B4371290C7
:1005FE000044E0900035F0900045E090003EF08021
:10060E000674039007B1F022E57A64046006E5995A
:10061E0064FF6002802AA2344004D2348020E57A3E
:10062E00600874E6257A900032F0757A00E57960FC
:10063E000874F02579900032F0757900C23480028A
:10064E00C234E57A9033F8F8282873757A00E59964
:10065E00B4FF03757901E599B4FE03757902E59946
:10066E00B4FD03757903E599B4FC03757904E59936
:10067E00B4FA03757905E599B4FB06757A01123B58
:10068E009FE599B4F906757A04123B9FE599D394C8
:10069E00E54007E599C394F04002801685997B7575
:1006AE007A027E017F00E57BC394E61261D88E5EEE
:1006BE008F5F9007A9E4F0A3F0E599D394C44007A7
:1006CE00E599C394E64002802885997B757A037478
:1006DE00E5C3957BF55F755E00AE5EAF5F905BD454
:1006EE001261A7E493F87401939007A9C8F0A3C808
:1006FE00F0D299020AB3900044E070429007A9E04C
:10070E00FEA3E0FF74FFBE00039F5009EFC39446A3
:10071E00EE940640119007A9E0FEA3E0FFEFD394FC
:10072E006DEE940640139007A9E0FEA3E0FF900043
:10073E00651261FFE599F08003859953801190074A
:10074E00A9E0FEA3E0FF9000651261FFE599F0902D
:10075E0007A91261E69007A9E0FEA3E0FFEFB4013E
:10076E0006EEB40702800302089B900765E0B43CD6
:10077E00028003020885C29C900044E0900103F0C1
:10078E00900045E0900072F0900046E0900092F0EC
:10079E00900047E09000BBF0900048E0900067F0BA
:1007AE00900049E09000ADF090004AE09000CBF050
:1007BE0090004BE090009FF090004CE09000BDF058
:1007CE0090004DE09000EDF012367F900056E090D4
:1007DE0000D4F0900057E090008BF0900058E0901D
:1007EE00008CF074639007A5F8E4F0E8A3F074AB06
:1007FE0090002FF012044890002FE4F075096475F4
:10080E0008001200E3A21D4038755201E552D39440
:10081E0007502CE5529007A5F8E4F0E8A3F074AA6F
:10082E0090002FF012010FE552C39407500975097D
:10083E00647508001200E37852740126F650CD80DC
:10084E0036755208E552D3940E502CE5529007A5FA
:10085E00F8E4F0E8A3F074AA90002FF012010FE56F
:10086E0052C3940E50097509647508001200E3789E
:10087E0052740126F650CD74C89007A5F8E4F0E83E
:10088E00A3F0D29C757A007579007599FB020AB3B4
:10089E009007A9E0FEA3E0FFEF4E700685995D7507
:1008AE005C009007A9E0FEA3E0FF74016F4E701B81
:1008BE00AC5CAD5DAA5EAB5FED2BFBEC3AFA8A0643
:1008CE008B079000651261FFE599F09007A9126100
:1008DE00E69007A9E0FEA3E0FF74026F4E7021AC14
:1008EE005CAD5D74566D4C7006E57B64E66002800F
:1008FE0003123B9F12367F857B99757A00757900BE
:10090E00020AB39007A9E0FEA3E0FF900065126112
:10091E00FFE599F09007A91261E69007A9E0FEA302
:10092E00E0FFAC5EAD5F8F028E038C068D07905C90
:10093E00161261A7E493F9740193FEEAD39EEB9924
:10094E004009857B99757A00757900020AB3900784
:10095E00A9E0FEA3E0FF9000651261FFE599F0901B
:10096E0007A91261E69007A9E0FEA3E0FFEFB4002D
:10097E0006EEB401028003020AB390003DE075F06A
:10098E0002A4FDACF08D52ED90006512620AEDFAF4
:10099E00E0FBEA90006812620AEBFAE0FBEA2BFA3F
:1009AE0090003DE0B502028003020AA50DED900015
:1009BE006512620AE552FDE0FAED90006912620AD4
:1009CE00EAFDE0FAEDC39AFD90003DE0B505028028
:1009DE0003020AA5E55290006712620AE552FDE095
:1009EE00FAED90006A12620AEAFDE0FAED2AFD9035
:1009FE00003DE0B505028003020AA5E55290006BAA
:100A0E0012620AFDE0FAED90003DE0F4042A900037
:100A1E0044F0E55290006C12620AFDE0FAED90008F
:100A2E003DE0F4042A900045F0E55290006D12620C
:100A3E000AFDE0FAED90003DE0F4042A900046F045
:100A4E00E55290006E12620AFDE0FAED90003DE074
:100A5E00F4042A9007A5F8E4F0E8A3F074AB900034
:100A6E002FF01204487509647508001200E3900710
:100A7E00A51261E61204487509647508001200E3B8
:100A8E009007A51261E61204487599F97509647507
:100A9E0008001200E380FE7599FF75096475080061
:050AAE001200E380FED0
:0F33F80002065902070402089E02091102095C2D
:100AB30022E579903407F8282873020B989007A948
:100AC300E0FEA3E0FF9000331261FFE0F599900789
:100AD300A91261E69007A9E0FEA3E0FF74116F4E2F
:100AE3007003757900020B98854B99020B98900758
:100AF300A9E0FEA3E0FF9000651261FFE0F599EF26
:100B0300B40107EEB407037579009007A91261E6F3
:070B1300020B989007AAE015
:0F340700020ABD020AC0020AEB020AF1020B160A
:100B1A009035BAF8282873852A998067853C998088
:100B2A0062853E99805D85429980588544998053B3
:100B3A00854599804E854699804985479980449094
:100B4A000012E0F599803CA235B340077599FAC2C4
:100B5A00358017A226B3400575990F800B90003295
:100B6A00E0F599900032E4F0C22680178548998012
:100B7A0012854399800D85499980087599FC8003EF
:030B8A007579007A
:1035BA00020B21020B26020B2B020B30020B3502E7
:1035CA000B3A020B3F020B44020B49020B51020B4E
:0D35DA0076020B7B020B80020B85020B8A30
:0B0B8D009007A91261E680031235E713
:03341600020B9511
:100B980022E5632538FFAE3750010E9000651261DB
:100BA800FFE0F564E5632538FFAE3750010E0FBF4F
:100BB80000010E9000651261FFE0F565856B67E541
:100BC80064B565058564638041E565D39564401D1A
:100BD800E565C395648566F0A4FFAEF0E5678E040D
:100BE8008F05FF1261C8ED2564F563801DE564C3B8
:100BF80095658566F0A4FFAEF0E5678E048F05FF66
:100C08001261C8EDF4042564F56322E565D39564A3
:100C1800401DE565C395648566F0A4FFAEF0E56701
:100C28008E048F05FF1261C8ED2564F563801DE50C
:100C380064C395658566F0A4FFAEF0E5678E048F02
:100C480005FF1261C8EDF4042564F5632290006B7A
:100C5800E0B40170E54475F00A84FF7E008F63E517
:100C68004475F00A84ADF07C008D66756B0A7537A3
:100C780005753824E563C394115005120B99800655
:100C880090059AE0F563E56390005BF0E54475F044
:100C98000A84FF7E008F63E54475F00A84ADF07C1A
:100CA800008D66756B0A75370575385AE563C39408
:100CB800115005120B9980069005D0E0F563E563A5
:100CC80090000AF02290006BE0B4016AE54475F0E8
:100CD8000A84FF7E008F63E54475F00A84ADF07CDA
:100CE800008D66756B0A753705753836E563C394EC
:100CF800115005120B9980069005ACE0F5638563E9
:100D080077E54475F00A84FF7E008F63E54475F04B
:100D18000A84ADF07C008D66756B0A7537057538E9
:100D280048E563C394115005120B9980069005BEDF
:100D3800E0F56385637822E53C75F00484FF7E0066
:100D48008F63E53C75F00484ADF07C008D66756BAF
:100D580004753701753800E563C3943F5005120BDD
:100D68009980069001A4E0F5638563557554009059
:100D78000031E075F020A4FFAEF09000B6E08E04DC
:100D88008F05FF1261C88D6390009EE0D3953C509B
:100D980003020E459000C2E0D3953C4010ED90014F
:100DA800A512620AE0F557755600020E4290008DB2
:100DB800E0D3953C4043E5639001A512620AE0F553
:100DC80064E5639001C512620AE0F5659000C2E02F
:100DD800F404253CF56690008DE0FE9000C2E0F436
:100DE800042EF567E564B565058564638003120C18
:100DF800138563577556008041E5639001C51262FB
:100E08000AE0F564E5639001E512620AE0F5659091
:100E1800008DE0F404253CF56690009EE0FE90000D
:100E28008DE0F4042EF567E564B565058564638097
:100E380003120C13856357755600020EEC9000C51B
:100E4800E0D3953C5011E56390022512620AE0F563
:100E580057755600020EEC90008EE0D3953C504337
:100E6800E56390020512620AE0F564E563900225E5
:100E780012620AE0F56590008EE0F404253CF56600
:100E88009000C5E0FE90008EE0F4042EF567E5645E
:100E9800B565058564638003120C13856357755621
:100EA800008041E5639001E512620AE0F564E563BC
:100EB80090020512620AE0F56590009EE0F40425B0
:100EC8003CF56690008EE0FE90009EE0F4042EF55E
:100ED80067E564B565058564638003120C13856353
:100EE80057755600229000D6E0F568756B11753776
:100EF80002753800AE29AF2AE56875F00FA4FDAC7D
:100F0800F0EDD39FEC9E4021E5688E048F05FF121B
:100F180061C8ED75F010A4FFAEF0E53C75F01184E2
:100F2800FD7C00ED2FF569800EE53C75F01184FF1E
:100F38007E00EF24F0F569856963E53C75F011845E
:100F4800AFF07E008F66120B9985636AAE29AF2ACF
:100F58009000D6E075F00FA4FDACF0EDD39FEC9EA9
:100F68004028753702753810856963120B99856AB0
:100F780064856365AE29AF2AE5688E048F05FF1284
:100F880061F38D66856867120C1385635575540087
:100F9800755764755600229000D6E0F568756B1198
:100FA800753702753800AE29AF2AE56875F00FA4C9
:100FB800FDACF0EDD39FEC9E4021E5688E048F05D3
:100FC800FF1261C8ED75F010A4FFAEF0E53E75F0B4
:100FD8001184FD7C00ED2FF569800EE53E75F0115A
:100FE80084FF7E00EF24F0F569856963E53E75F0BE
:100FF8001184AFF07E008F66120B9985636AAE2963
:10100800AF2A9000D6E075F00FA4FDACF0EDD39FA9
:10101800EC9E4028753702753810856963120B9964
:10102800856A64856365AE29AF2AE5688E048F05F5
:10103800FF1261F38D66856867120C138563557519
:1010480054009000A0E0B40453E53C75F00484FF1C
:101058007E008F63E53C75F00484ADF07C008D66FE
:10106800756B04753701753800E563C3943F500507
:10107800120B9980069001A4E0F563AE54AF55E5D4
:10108800631261D874648E048F05FF1261C8AE5470
:10109800AF55EF2DFDEE3CFC8C548D55755764759E
:1010A80056002290006BE0B40146E54475F00A84CE
:1010B800FF7E008F63E54475F00A84ADF07C008DF7
:1010C80066756B0A753705753800E563C39411506A
:1010D80005120B998006900576E0F563AE56AF577A
:1010E800E5632FFF50010E746412621C8E568F57F1
:1010F80090006CE0B40146E54575F00A84FF7E0077
:101108008F63E54575F00A84ADF07C008D66756BDC
:101118000A75370575386CE563C394115005120BD1
:101128009980069005E2E0F563AE56AF57E5632F68
:10113800FF50010E746412621C8E568F5790007B0C
:10114800E0B40249E547C3944175F00584FF7E0089
:101158008F63E54775F00584ADF07C008D66756B8F
:1011680005753706753800E563C394135005120BEF
:10117800998006900678E0F563AE56AF57E5632F81
:10118800FF50010E746412621C8E568F579000BD7A
:10119800E0B40202800302124AE53C75F01584FFB0
:1011A8007E008F63E53C75F01584ADF07C008D669C
:1011B800756B157537037538F4E563C3940B5005E3
:1011C800120B998006900464E0F563E56375F0FFFF
:1011D800A4FFAEF09000BEE08E048F05FF1261C838
:1011E800ED900054F0E54375F078A4FFAEF074FF7D
:1011F8008E048F05FF1261C88C378D3874028C06F7
:101208008D071200398F63AC37AD387404FF126153
:10121800F38D66756B04753706753828E563C394D6
:101228001D5005120B9980069006AAE0F563AE568C
:10123800AF57E5632FFF50010E746412621C8E567F
:101248008F5790006AE0B4025DE53E75F064A4FF34
:10125800AEF074081200398E398F3A74058E048FF7
:1012680005FF1261C88D63AE39AF3A74058E048FDD
:1012780005FF1261F38D66756B057537057538DEE8
:10128800E563C394135005120B998006900656E047
:10129800F563AE56AF57E5632FFF50010E74641225
:1012A800621C8E568F579000ACE0703C900031E085
:1012B80075F00584FF7E008F63900031E075F005BE
:1012C80084ADF07C008D66756B057537057538C083
:1012D800E563C3941D5005120B998006900642E001
:1012E800F563E56390005CF022900073E0B40117A9
:1012F8009007ACE02557FFAE5650010E9000C7E0AE
:1013080012621C8E568F579000EBE0B401149000C7
:10131800ECE0A829B80004952A5007E53CC3953DA0
:1013280040028012900095E02557FFAE5650010EFE
:101338008E568F57802F900073E0B40316A228B3FF
:10134800B350109007AFE0C39405A829B8000695DC
:101358002A40028010900095E02557FFAE565001B4
:101368000E8E568F5790006DE0B40202800302156E
:101378004D900070E0602FE544D3944640289000DB
:101388000BE0FEA3E0FF9000ABE075F003A4FDAC1A
:10139800F0EFD39DEE9C400E9000CFE0A829B80056
:1013A80005D3952A500302154D9000B8E0853CF00E
:1013B800A4FFAEF074051261D874071200398E3795
:1013C8008F38900077E0A829B80004952A50129029
:1013D8000078E075F002A4FDACF0EFC39DEE9C40F0
:1013E8000302154DE53C75F00B84FF7E009005F572
:1013F8001261FFFEE0FFEE90006FE0FEEF8E0088C6
:10140800F0A4FFAEF074648E048F05FF1261C88CDF
:10141800378D38900031E075F018A4FFAEF09000D9
:10142800B6E08E048F05FF1261C88C068D07900602
:101438000D1261FFAE37AF38E01261D874648E04C4
:101448008F05FF1261C88C378D38E542A837B80080
:1014580077D395384072E542C39538FFE49537FE57
:101468008E378F387428BE00039F500C7538287546
:101478003700740D900032F0AE37AF38900070E04E
:101488001261D874288E048F05FF1261C88C378DBD
:1014980038AE54AF55740A8E048F05FF1261C88D9B
:1014A800068C07AC37AD38CFCECF120003740A8E46
:1014B800048F05FF1261C88C378D38AE54AF5512B2
:1014C80062248E548F55807DE542A837B800049574
:1014D800385072AE37AF38E54212621C8E378F38FB
:1014E8007428BE00039F500C753828753700740D9A
:1014F800900032F0AE37AF38900070E01261D874C7
:10150800288E048F05FF1261C88C378D38AE54AF12
:1015180055740A8E048F05FF1261C88D068C07ACBE
:1015280037AD38CFCECF120003740A8E048F05FF73
:101538001261C88C378D38AE54AF55EF2DFDEE3C97
:10154800FC8C548D55229000CBE0B4026AE53C75C2
:10155800F00884FF7E008F63E53C75F00884ADF0E9
:101568007C008D66756B087537017538E0E563C3D7
:10157800943F5005120B998006900264E0F563854C
:101588006359755800AE58AF59AC56AD57120003A1
:1015980074648E048F05FF1261C88C588D599000B1
:1015A80068E08C068D071261D874648E048F05FF7D
:1015B8001261C88C588D59AE54AF55AC56AD571200
:1015C800000374648E048F05FF1261C88C548D5516
:1015D800900068E08C068D071261D874648E048FC1
:1015E80005FF1261C88C548D55A20D401DAE29AF60
:1015F8002A7405BE00039F5002D20DE53ED394CC59
:101608004008D2017411900032F09000CAE0B40290
:10161800089000CCE0640160028035AE54AF55E517
:10162800481261D874E78E048F05FF1261C88C5484
:101638008D559000CBE0B40217AE58AF59E548126B
:1016480061D874E78E048F05FF1261C88C588D59D4
:1016580090008AE05402601B900081E0A829B8003D
:1016680012D3952A400DA20DB3B35007E53EC3949B
:101678009A40028028AE61AF6290007FE075F00268
:10168800A4FDACF0EF2DFDEE3CFC74022DFD5001E5
:101698000CE53EBC0007D39D4003756F01853E6293
:1016A800756100E56F70030217919000DDE0C39546
:1016B8006F50030217839000EDE0C394025076E563
:1016C8004475F00A84FF7E009005651261FFE0F51D
:1016D80038753700AE37AF38900080E01261D874A3
:1016E800648E048F05FF1261C88C398D3A9000DD35
:1016F800E004C3956F8C068D071261D89000DDE079
:101708008E048F05FF1261C88C398D3AAE54AF55DF
:10171800EF2DFDEE3CFC8C548D559000CBE0B402CF
:1017280012AE58AF59AA39AB3AEF2BFBEE3AFA8A08
:10173800588B5980469000DDE004C3956F8577F09B
:10174800A4FFAEF09000DDE08E048F05FF1261C8A3
:101758008C398D3AAE54AF55EF2DFDEE3CFC8C54D0
:101768008D559000CBE0B40212AE58AF59AA39ABF0
:101778003AEF2BFBEE3AFA8A588B59056F9000DD49
:10178800E0C3956F5003756F0090008AE0540160C4
:101798001B90007EE0A829B80012D3952A400DA21C
:1017A8000DB3B35007E53CC394CC400280259000AC
:1017B8007CE075F003A4FFAEF0E56C2FFF50010E3E
:1017C80074032FFF50010EE53CBE0007D39F400372
:1017D800757001853C6CE57070030218C49000DEDA
:1017E800E0C3957050030218B69000EDE0C3940270
:1017F8005076E54475F00A84FF7E00900565126115
:10180800FFE0F538753700AE37AF3890007DE0124D
:1018180061D874648E048F05FF1261C88C398D3AC3
:101828009000DEE004C395708C068D071261D89095
:1018380000DEE08E048F05FF1261C88C398D3AAE48
:1018480054AF55EF2DFDEE3CFC8C548D559000CBDC
:10185800E0B40212AE58AF59AA39AB3AEF2BFBEEFF
:101868003AFA8A588B5980469000DEE004C3957096
:101878008578F0A4FFAEF09000DEE08E048F05FFBF
:101888001261C88C398D3AAE54AF55EF2DFDEE3C40
:10189800FC8C548D559000CBE0B40212AE58AF5971
:1018A800AA39AB3AEF2BFBEE3AFA8A588B590570F6
:1018B8009000DEE0C3957050037570009000E0E082
:1018C8002555FFAE5450010E8E548F5590008FE071
:1018D800A854B800049555500990008FE0F5557547
:1018E80054009000CBE0B4020D90008FE0A858B8E7
:1018F800000695594002800990008FE0F559755807
:1019080000229000CBE0B401028003021A15A20D58
:10191800B35003021A13900096E0B40168AE54AFB6
:1019280055AC29AD2A120003743C8E048F05FF12B2
:1019380061C89000A6E0BC00109D400D9000A8E092
:10194800A854B8000495555002D202AE54AF55AC15
:1019580029AD2A120003743C8E048F05FF1261C85A
:101968009000A6E0C3940ABC0015D39D40119000D6
:10197800A8E0C39405A854B80005D3955550028033
:1019880002C2028068AE54AF55AC29AD2A120003DA
:1019980074788E048F05FF1261C89000A6E0BC0021
:1019A800109D400D9000A8E0A854B800049555502B
:1019B80004D2028038AE54AF55AC29AD2A120003C8
:1019C80074788E048F05FF1261C89000A6E0C39456
:1019D8000ABC0015D39D40119000A8E0C39405A847
:1019E80054B80005D3955550028002C202A202B332
:1019F8004019AE54AF559000A7E01261D874648EB8
:101A0800048F05FF1261C88C548D558002C202A252
:101A180000B34006A201B3B35009900011E4F0A34B
:101A2800F08024AE54AF557400D39F74019E400CCF
:101A3800900011E554F0A3E555F0800B74FF900079
:101A480011F8E4F0E8A3F09000ADE0D39402400C64
:101A5800900098E07006A20DB3B34002801AAE540D
:101A6800AF5574021261D88E548F55AE58AF597461
:101A7800021261D88E588F59900096E0B4011AAEC0
:101A880054AF5574021261D88E548F55AE58AF5961
:101A980074021261D88E588F59AE54AF55745E12C5
:101AA80061D8740A8E048F05FF1261C88C548D5555
:101AB8009000CBE0B40217AE58AF59745E1261D8EB
:101AC800740A8E048F05FF1261C88C588D59AE5464
:101AD800AF557402BE000AD39F400675550275546F
:101AE80000AE58AF597402BE000AD39F400675591C
:101AF8000275580090000FE554F0A3E555F02290C8
:101B08000031E090036512620AE0F56D756E64902D
:101B18000031E0FE9000A1E0D39E4037E53C75F02F
:101B28000884FF7E008F63E53C75F00884ADF07C87
:101B3800008D66756B08753703753896E563C39431
:101B48001F5005120B99800690041AE0F56385630F
:101B58006E8035E53C75F00884FF7E008F63E53CB8
:101B680075F00884ADF07C008D66756B08753703D9
:101B78007538B6E563C3941F5005120B998006901B
:101B8800043AE0F56385636E229000D7E0F5687546
:101B98006B11753704753800AE29AF2AE56875F002
:101BA8000FA4FDACF0EDD39FEC9E4021E5688E04B8
:101BB8008F05FF1261C8ED75F010A4FFAEF0E53C8B
:101BC80075F01184FD7C00ED2FF569800EE53C75FC
:101BD800F01184FF7E00EF24F0F569856963E53C28
:101BE80075F01184AFF07E008F66120B9985636AD9
:101BF800AE29AF2A9000D7E075F00FA4FDACF0ED48
:101C0800D39FEC9E40287537047538108569631298
:101C18000B99856A64856365AE29AF2AE5688E04E9
:101C28008F05FF1261F38D66856867120C13856353
:101C38006D756E64229000D7E0F568756B11753785
:101C480004753800AE29AF2AE56875F00FA4FDAC1D
:101C5800F0EDD39FEC9E4021E5688E048F05FF12BE
:101C680061C8ED75F010A4FFAEF0E53E75F0118483
:101C7800FD7C00ED2FF569800EE53E75F01184FFBF
:101C88007E00EF24F0F569856963E53E75F01184FF
:101C9800AFF07E008F66120B9985636AAE29AF2A72
:101CA8009000D7E075F00FA4FDACF0EDD39FEC9E4B
:101CB8004028753704753810856963120B99856A51
:101CC80064856365AE29AF2AE5688E048F05FF1227
:101CD80061F38D66856867120C1385636D756E6494
:101CE8009000D2E0B40479900031E0FE9000A1E0C9
:101CF800D39E4037E53C75F00884FF7E008F63E58E
:101D08003C75F00884ADF07C008D66756B087537FE
:101D180003753896E563C3941F5005120B99800626
:101D280090041AE0F56385636E8035E53C75F0082C
:101D380084FF7E008F63E53C75F00884ADF07C007D
:101D48008D66756B087537037538B6E563C3941FE0
:101D58005005120B99800690043AE0F56385636E8E
:101D68002290006BE0B4013BE54475F00A84FF7EE5
:101D7800008F63E54475F00A84ADF07C008D6675CC
:101D88006B0A753705753812E563C394115005124F
:101D98000B998006900588E0F563E56E2563C3948A
:101DA80064F56E90006CE0B4013BE54575F00A847B
:101DB800FF7E008F63E54575F00A84ADF07C008DE9
:101DC80066756B0A75370575387EE563C3941150DF
:101DD80005120B9980069005F4E0F563E56E25631E
:101DE800C39464F56EE56D256EF560900073E0B4FC
:101DF80002109007ABE02560FE9000C7E0F4042EC7
:101E0800F5609000CAE0D394014040E548C394E7E8
:101E1800501D74E7C39548FE9007ADE08E00F5F0BD
:101E2800E884FF7E008F63E5602563F560801CE52C
:101E380048C394E7FE9007ADE08E00F5F0E884FF14
:101E48007E008F63E560C39563F560A20D4006E5EB
:101E58006D2464F560E560D394644009E560C3943B
:101E680064F56080037560009000A3E0C39560503E
:101E7800069000A3E0F56022D20090005AE0A8295D
:101E8800B80004952A504190005AE0A829B80004E7
:101E9800952A500375600F90005AE004A829B800ED
:101EA80004952A500375600A90005AE02402A82974
:101EB800B80004952A5005756005C20090005AE0E4
:101EC80060067409900032F0C2387E017F009000ED
:101ED800A9E01261D89000B8E08E048F05FF126166
:101EE800C8E53CBC0017D39D40139000B2E0B40293
:101EF80004D2388002C200740A900032F09000AA1E
:101F0800E0C3954450159000BCE0A829B80004959A
:101F18002A5002C200740B900032F0E544C3946466
:101F2800501D900102E0600D900102E0A829B80060
:101F380006952A40028008C200740B900032F0A275
:101F48000040037560059000EBE0B401149000ECCC
:101F5800E0A829B80004952A5007E53CC3953D4000
:101F6800028008900094E0F560803A900073E0B435
:101F78000306A228B3B34002802B9007AFE0C394B6
:101F880005A829B80004952A500C900094E0F56043
:101F9800740C900032F09007AFE0A829B8000495BF
:101FA8002A5002C200856049900065E02560FE90D5
:101FB8000031E075F01E84FC7F00EE2CF560229065
:101FC8000031E075F00584FF7E008F63900031E0FA
:101FD80075F00584ADF07C008D66756B057537036B
:101FE8007538D69000B6E01475F00584FF7E00E5DC
:101FF80063BE00039F5005120B99800BE5639004A4
:102008003B12620AE0F563E5639007AEF09007AE15
:10201800E0FE9000A5E0C39E50089000A5E0900760
:10202800AEF022E54475F00A84FF7E009005651243
:1020380061FFE0F572E572D394644010E572C394D1
:102048006475F00F84FF7E008F72800375720090B4
:102058000088E02572F5722290079FE0FEA3E0FF5A
:102068007404120039E53C1261D8740F8E048F0590
:10207800FF1261C890079DECF0A3EDF090007BE0A3
:10208800B40262E547C3944175F00584FF7E008F72
:1020980063E54775F00584ADF07C008D66756B05CA
:1020A800753706753814E563C394175005120B99F4
:1020B800800690068CE0F56390079DE0FEA3E0FFA4
:1020C800740A8E048F05FF1261C8E5638C068D07BC
:1020D8001261D8740A8E048F05FF1261C890079D9B
:1020E800ECF0A3EDF090079DE0FEA3E0FF9007A3BE
:1020F800E0FCA3E0FDEDD39FEC9E400F9007A3E02A
:10210800F8A3E090079DC8F0A3C8F0229006ACE0C1
:10211800903419F8282873804C852A5280479000FB
:10212800B8E0853CF0A4FFAEF074081200398F5275
:102138008033853E52802E854452802985455280C1
:1021480024854652801F854752801A85485280153B
:102158008543528010854252800B854952800690F3
:052168000012E0F55239
:1034190002211F02212102212602213A02213F0213
:10342900214402214902214E02215302215802213D
:073439005D02216202216720
:10216D009006ADE0FE9006AEE0D39E404B9006ACDF
:10217D00E0B404189006AEE0C395525002D22990F7
:10218D0006ADE0D395524002C229802A9006ADE0FB
:10219D00C3955250099006AEE0D39552500280027D
:1021AD00D2299006ADE0D3955250099006AEE0C30A
:1021BD0095525002C229802A9006ADE0D395524027
:1021CD00099006AEE0C3955240028002C2299006E6
:1021DD00ADE0C3955240099006AEE0D39552400252
:1021ED00D229229006B0E0903440F8282873804C14
:1021FD00852A5280479000B8E0853CF0A4FFAEF0F0
:10220D0074081200398F528033853E52802E8544DA
:10221D005280298545528024854652801F8547521C
:10222D00801A854852801585435280108542528010
:0C223D000B8549528006900012E0F5521B
:103440000221FB0221FD02220202221602221B029D
:10345000222002222502222A02222F0222340222C4
:073460003902223E02224363
:102249009006B1E0FE9006B2E0D39E405F9006B0E2
:10225900E0B404189006B2E0C395525002D22A9015
:1022690006B1E0D395524002C22A803E9006B1E001
:10227900C3955250099006B2E0D39552500280029C
:10228900D22A9006B1E0D3955250099006B2E0C324
:1022990095525002C22A9006B0E0B401099000C4D8
:1022A900E0D3953E50028002C22A802A9006B1E00E
:1022B900D3955240099006B2E0C39552400280027C
:1022C900C22A9006B1E0C3955240099006B2E0D304
:1022D90095524002D22A229006B4E0903467F82839
:1022E9002873804C852A5280479000B8E0853CF0DD
:1022F900A4FFAEF074081200398F528033853E5224
:10230900802E8544528029854552802485465280F5
:102319001F854752801A854852801585435280107F
:10232900854252800B8549528006900012E0F55291
:103467000222EB0222ED0222F202230602230B02C2
:10347700231002231502231A02231F0223240223E7
:073487002902232E0223336A
:102339009006B5E0FE9006B6E0D39E404B9006B4F9
:10234900E0B404189006B6E0C395525002D22B901F
:1023590006B5E0D395524002C22B802A9006B5E01B
:10236900C3955250099006B6E0D3955250028002A7
:10237900D22B9006B5E0D3955250099006B6E0C32A
:1023890095525002C22B802A9006B5E0D39552404F
:10239900099006B6E0C3955240028002C22B90060E
:1023A900B5E0C3955240099006B6E0D39552400274
:1023B900D22B229006B8E090348EF8282873804CEE
:1023C900852A5280479000B8E0853CF0A4FFAEF022
:1023D90074081200398F528033853E52802E85440D
:1023E9005280298545528024854652801F8547524F
:1023F900801A854852801585435280108542528043
:0C2409000B8549528006900012E0F5524D
:10348E000223C70223C90223CE0223E20223E7024C
:10349E0023EC0223F10223F60223FB022400022472
:0734AE000502240A02240FAD
:102415009006B9E0FE9006BAE0D39E404B9006B810
:10242500E0B404189006BAE0C395525002D22C903D
:1024350006B9E0D395524002C22C802A9006B9E035
:10244500C3955250099006BAE0D3955250028002C6
:10245500D22C9006B9E0D3955250099006BAE0C344
:1024650095525002C22C802A9006B9E0D39552406D
:10247500099006BAE0C3955240028002C22C90062C
:10248500B9E0C3955240099006BAE0D3955240028F
:10249500D22C229006BCE09034B5F8282873804CE5
:1024A500852A5280479000B8E0853CF0A4FFAEF045
:1024B50074081200398F528033853E52802E854430
:1024C5005280298545528024854652801F85475272
:1024D500801A854852801585435280108542528066
:0C24E5000B8549528006900012E0F55271
:1034B5000224A30224A50224AA0224BE0224C302D4
:1034C50024C80224CD0224D20224D70224DC0224FB
:0734D500E10224E60224EBF2
:1024F1009006BDE0FE9006BEE0D39E404B9006BC28
:10250100E0B404189006BEE0C395525002D22D905B
:1025110006BDE0D395524002C22D802A9006BDE04F
:10252100C3955250099006BEE0D3955250028002E5
:10253100D22D9006BDE0D3955250099006BEE0C35E
:1025410095525002C22D802A9006BDE0D39552408B
:10255100099006BEE0C3955240028002C22D90064A
:10256100BDE0C3955240099006BEE0D395524002AA
:10257100D22D229006C0E09034DCF8282873804CDC
:10258100852A5280479000B8E0853CF0A4FFAEF068
:1025910074081200398F528033853E52802E854453
:1025A1005280298545528024854652801F85475295
:1025B100801A854852801585435280108542528089
:0C25C1000B8549528006900012E0F55294
:1034DC0002257F02258102258602259A02259F025C
:1034EC0025A40225A90225AE0225B30225B8022582
:0734FC00BD0225C20225C735
:1025CD009006C1E0FE9006C2E0D39E404B9006C03F
:1025DD00E0B404189006C2E0C395525002D22E907A
:1025ED0006C1E0D395524002C22E802A9006C1E06A
:1025FD00C3955250099006C2E0D395525002800205
:10260D00D22E9006C1E0D3955250099006C2E0C378
:10261D0095525002C22E802A9006C1E0D3955240A9
:10262D00099006C2E0C3955240028002C22E900668
:10263D00C1E0C3955240099006C2E0D395524002C5
:10264D00D22E229006C4E0903503F8282873804CD2
:10265D00852A5280479000B8E0853CF0A4FFAEF08B
:10266D0074081200398F528033853E52802E854476
:10267D005280298545528024854652801F854752B8
:10268D00801A8548528015854352801085425280AC
:0C269D000B8549528006900012E0F552B7
:1035030002265B02265D02266202267602267B02E3
:10351300268002268502268A02268F022694022608
:073523009902269E0226A377
:1026A9009006C5E0FE9006C6E0D39E404B9006C456
:1026B900E0B404189006C6E0C395525002D22F9098
:1026C90006C5E0D395524002C22F802A9006C5E084
:1026D900C3955250099006C6E0D395525002800224
:1026E900D22F9006C5E0D3955250099006C6E0C393
:1026F90095525002C22F802A9006C5E0D3955240C8
:10270900099006C6E0C3955240028002C22F900686
:10271900C5E0C3955240099006C6E0D395524002E0
:10272900D22F229006C8E090352AF8282873804CC9
:10273900852A5280479000B8E0853CF0A4FFAEF0AE
:1027490074081200398F528033853E52802E854499
:102759005280298545528024854652801F854752DB
:10276900801A8548528015854352801085425280CF
:0C2779000B8549528006900012E0F552DA
:10352A0002273702273902273E022752022757026B
:10353A00275C02276102276602276B02277002278F
:07354A007502277A02277FBA
:102785009006C9E0FE9006CAE0D39E404B9006C86D
:10279500E0B404189006CAE0C395525002D23090B6
:1027A50006C9E0D395524002C230802A9006C9E09E
:1027B500C3955250099006CAE0D395525002800243
:1027C500D2309006C9E0D3955250099006CAE0C3AD
:1027D50095525002C230802A9006C9E0D3955240E6
:1027E500099006CAE0C3955240028002C2309006A5
:1027F500C9E0C3955240099006CAE0D395524002FC
:10280500D230229006CCE0903551F8282873804CC0
:10281500852A5280479000B8E0853CF0A4FFAEF0D1
:1028250074081200398F528033853E52802E8544BC
:102835005280298545528024854652801F854752FE
:10284500801A8548528015854352801085425280F2
:0C2855000B8549528006900012E0F552FD
:1035510002281302281502281A02282E02283302F3
:10356100283802283D02284202284702284C022816
:073571005102285602285BFD
:102861009006CDE0FE9006CEE0D39E404B9006CC84
:10287100E0B404189006CEE0C395525002D23190D4
:1028810006CDE0D395524002C231802A9006CDE0B8
:10289100C3955250099006CEE0D395525002800262
:1028A100D2319006CDE0D3955250099006CEE0C3C7
:1028B10095525002C231802A9006CDE0D395524004
:1028C100099006CEE0C3955240028002C2319006C3
:1028D100CDE0C3955240099006CEE0D39552400217
:1028E100D231229006D0E0903578F8282873804CB8
:1028F100852A5280479000B8E0853CF0A4FFAEF0F5
:1029010074081200398F528033853E52802E8544DF
:102911005280298545528024854652801F85475221
:10292100801A854852801585435280108542528015
:0C2931000B8549528006900012E0F55220
:103578000228EF0228F10228F602290A02290F027E
:10358800291402291902291E02292302292802299D
:073598002D02293202293740
:10293D009006D1E0FE9006D2E0D39E404B9006D09B
:10294D00E0B404189006D2E0C395525002D23290F2
:10295D0006D1E0D395524002C232802A9006D1E0D2
:10296D00C3955250099006D2E0D395525002800281
:10297D00D2329006D1E0D3955250099006D2E0C3E1
:10298D0095525002C232802A9006D1E0D395524022
:10299D00099006D2E0C3955240028002C2329006E1
:1029AD00D1E0C3955240099006D2E0D39552400232
:1029BD00D23222AE5AAF5B74F5D39F74019E40089C
:1029CD00785A12622C022ADA755B01755A00AE290B
:1029DD00AF2AE572BE000DD39F400990009AE0D357
:1029ED00957340028023757300E572C3952AF552E5
:1029FD0090009DE0D395714008E5712552F57180E9
:102A0D000690009DE0F57180020573900076E0D38D
:102A1D00953E401CE53CC3953D4015AE29AF2AE5DA
:102A2D0072BE00039F500990009BE0D39574400245
:102A3D00806E9007B2E0A829B80004952A5003755E
:102A4D0076009007B2E0A829B8000BD3952A40066E
:102A5D00E52A9007B2F0E5767041E52AC39572F547
:102A6D0052E552D39405400375520590009CE0C386
:102A7D0095715007E552C3957140028009E571C308
:102A8D009552F571800690009CE0F57190009CE0E8
:102A9D00D39571400690009CE0F57175740080022D
:102AAD000574E5767016900076E0C3953E500DE501
:102ABD00722405A829B80006952A4002800F9000BF
:102ACD0089E0F57175760174789007B2F022AE5AEF
:102ADD00AF5B74E9D39F74039E4008785A12622C41
:102AED00022C79755B01755A00757132A233402A3B
:102AFD00757119900089E075F002A4FFAEF0E573D1
:102B0D00BE0006D39F4002D23305737576037478E9
:102B1D009007B2F0757500022C68AE29AF2AE572E8
:102B2D006F4E7003022C68E572BE000DD39F4009F5
:102B3D0090009AE0D395734002800F757300E5768F
:102B4D00C394035003757119800DE572C3952AF571
:102B5D0052E5732552F573900076E0D3953E400E05
:102B6D009007B2E0A829B80007D3952A4002800C3F
:102B7D000575900089E0B57503757600E576B403AB
:102B8D0006A20DB3B34002800A0575E575B43C038A
:102B9D00757602E576B402299007B2E0A829B8004F
:102BAD000ED3952A4009E52A9007B2F0757500906D
:102BBD000076E0C3953E500975750074789007B2A4
:102BCD00F0E576705A900076E0D3953E401CE53CDA
:102BDD00C3953D4015AE29AF2AE572BE00039F5047
:102BED000990009BE0D395744002800875740075C0
:102BFD00714B8028E52AC39572F552E552D39405A1
:102C0D004003755205900076E0D3953E4008E5747B
:102C1D002552F5748006E5742406F574757500E586
:102C2D00767016900076E0C3953E500DE572240542
:102C3D00A829B80006952A40028003757601E5762D
:102C4D00B401187571190575900089E0B575067593
:102C5D00760275750074789007B2F0E57175F00A1B
:102C6D00A4FFAEF09007A7EEF0A3EFF022E54C9095
:102C7D00359FF828287390006EE07003022E28907F
:102C8D0000A4E0B401028003022D78900030E0B57D
:102C9D003B028003022D757E017F00E5BE1261D8D7
:102CAD00E5BD2FFF50010E8E378F3874101261D88D
:102CBD00900059E08E048F05FF1261C89007B3ECA8
:102CCD00F0A3EDF0E54860089000CAE064026002F0
:102CDD0080269000CCE0B4011F9007B3E0FEA3E086
:102CED00FF74E71261D8E5488E048F05FF1261C8A5
:102CFD009007B3ECF0A3EDF090006EE0B4022790D6
:102D0D0007B5E0FEA3E0FF9007B3E0FCA3E0FDEF05
:102D1D002DFDEE3CFC74018C068D071200399007D9
:102D2D00B3EEF0A3EFF09007B3E0FEA3E0FF900742
:102D3D00B5E0FCA3E0FDEDD39FEC9E4004D23680C0
:102D4D0002B2369007B3E0F8A3E09007B5C8F0A340
:102D5D00C8F09000A0E064016006A236B3B3400253
:102D6D0080069007B4E0F53C022E26D2367E017F18
:102D7D0000E5BE1261D8E5BD2FFF50010E8E378FD5
:102D8D003874101261D8900059E08E048F05FF122F
:102D9D0061C89007B3ECF0A3EDF0E5486008900032
:102DAD00CAE06402600280269000CCE0B4011F905E
:102DBD0007B3E0FEA3E0FF74E71261D8E5488E0487
:102DCD008F05FF1261C89007B3ECF0A3EDF09000F2
:102DDD006EE0B402279007B5E0FEA3E0FF9007B3C5
:102DED00E0FCA3E0FDEF2DFDEE3CFC74018C068DA7
:102DFD00071200399007B3EEF0A3EFF09007B3E0A0
:102E0D00F8A3E09007B5C8F0A3C8F09000A0E06467
:102E1D000160069007B4E0F53C8003753C0090001E
:102E2D006AE07006754C01022C7A75BB180233F3FB
:102E3D0090006AE07003022FC97E017F00E5BE128B
:102E4D0061D8E5BD2FFF50010E8E378F389000B041
:102E5D00E0B4010F7E0F7FFFAC37AD381262248EC8
:102E6D00378F389000D5E0B40245AE37AF389000BB
:102E7D001BE0FCA3E0FDEDD39FEC9E400A90001BF0
:102E8D00E537F0A3E538F0AE37AF3890001DE0FC24
:102E9D00A3E0FDEFD39DEE9C400A90001DE537F0B9
:102EAD00A3E538F0AE37AF3874041200398F3E9079
:102EBD0000D5E0704CAE37AF3890001BE0FCA3E0BE
:102ECD00FDEFD39DEE9C40091262248E378F388022
:102EDD0006753800753700AE37AF3874101261D8EB
:102EED00900056E08E048F05FF1261C88C378D3827
:102EFD0074FFBC0009D39D400585383E8003753EA7
:102F0D00FE9000A0E0B401028003022FC7A20DB312
:102F1D00B3500E900074E0A829B80005D3952A503F
:102F2D0003022FBC900075E075F019A4FFAEF09070
:102F3D0000B8E08E048F05FF1261C89000B1E085E6
:102F4D003EF0A4FFAEF074648D028C038E048F05E9
:102F5D00FF1261C8EA2DFDEB3CFC8C378D38E5483E
:102F6D00600F9000CAE0B402089000CCE0640160EC
:102F7D00028017AE37AF3874E71261D8E5488E047A
:102F8D008F05FF1261C88C378D38AE37AF3890077B
:102F9D00B3E0FCA3E0FDEDD39FEC9E400585383CEE
:102FAD00800BA236B340069007B4E0F53C800BA22F
:102FBD0036B340069007B4E0F53C8003753E0090B3
:102FCD00006DE07006754C02022C7A75BB19023348
:102FDD00F390006DE0700302307EE53BD395284001
:102FED000302307C900019E0FEA3E0FFE54212627F
:102FFD001C900019EEF0A3EFF07E017F00E5BE12EC
:10300D0061D8E5BD2FFF50010E8E378F389000DA55
:10301D00E07013740A1261D874518E048F05FF127B
:10302D0061C88D428019AE37AF38740A1261D88FDE
:10303D00048E057E017F95CDCCCD1260C68F42E505
:10304D0042D394644003754264900019E0FEA3E0FE
:10305D00FFE5422FFF50010E900019EEF0A3EFF0A7
:10306D00900071E0048E048F05FF1261C88D4280BF
:10307D00037542329000BDE07006754C03022C7A48
:10308D0075BB130233F39000BDE0604A7E017F00F3
:10309D00E5BE1261D8E5BD2FFF50010E8E378F387A
:1030AD0074041200398F439000BFE08543F0A4FDF6
:1030BD00ACF07464FF1261C88D439000BEE085438F
:1030CD00F0A4FFAEF074FF8E048F05FF1261C8ED02
:1030DD00900055F0800375430090006BE07006750D
:1030ED004C04022C7A75BB170233F390006BE0B4DD
:1030FD000102800302318C7E017F00E5BE1261D892
:10310D00E5BD2FFF50010E8E378F389007B7E06069
:10311D00199007B7E014905C5812008CE493FC747E
:10312D000193FDEDC39FEC9E400280069007B7E032
:10313D0014F09007B7E0C394B3501DAE37AF38907D
:10314D0007B7E004905C5812008CE493FC74019373
:10315D00FDEFC39DEE9C400280069007B7E004F0A2
:10316D009007B7E0FE900091E08E0088F0A4FFAECE
:10317D00F074648E048F05FF1261C88D4480037551
:10318D00440090006CE07006754C05022C7A75BBFE
:10319D00160233F390006CE0B40102800302323565
:1031AD007E017F00E5BE1261D8E5BD2FFF50010EF7
:1031BD008E378F389007B8E060199007B8E01490FB
:1031CD005DC212008CE493FC740193FDEDC39FEC82
:1031DD009E400280069007B8E014F09007B8E0C357
:1031ED0094B3501DAE37AF389007B8E004905DC270
:1031FD0012008CE493FC740193FDEFC39DEE9C4093
:10320D000280069007B8E004F09007B8E0FE900049
:10321D0097E08E0088F0A4FFAEF074648E048F05E5
:10322D00FF1261C88D45800375450075BB1F0233C4
:10323D00F37E017F00E5BE1261D8E5BD2FFF500181
:10324D000E8E378F3874091261D874E68E048F058F
:10325D00FF1261C88D47900073E07006754C070230
:10326D002C7A75BB150233F3900073E070030233B3
:10327D008F7E017F00E5BE1261D8E5BD2FFF5001A5
:10328D000E8E378F3874041200398F46900073E01C
:10329D00B401159000C7E08546F0A4FFAEF07407A9
:1032AD00120039EF9007ACF0900073E0B402159066
:1032BD0000C7E08546F0A4FFAEF07407120039EFA9
:1032CD009007ABF0900073E0B40302800302338DDE
:1032DD009000B4E070389000C7E0601CE546C394E0
:1032ED00195002D228E546D394644002C2289000BA
:1032FD0093E09007AFF08014E546C394195002D2C5
:10330D0037E546D394324002C237C228806390001D
:10331D0093E070349000C7E08546F0A4FFAEF074E2
:10332D00FF8E048F05FF1261C8ED9007AFF0AE2937
:10333D00AF2A741EBE0006D39F4002D228E53ED3AD
:10334D0094E54002C2288029E546C3940A500DAE8B
:10335D0029AF2A741EBE0004D39F50028002D228CA
:10336D00E53ED394E54002C228900093E09007AF6C
:10337D00F09007AFE0C39405500674059007AFF0C9
:10338D0080037546009000CAE07006754C08022C4B
:10339D007A75BB1480509000CAE060397E017F00C1
:1033AD00E5BE1261D8E5BD2FFF50010E8E378F3867
:1033BD00EFD39421EE940E40057548FF8015AE377E
:1033CD00AF3874101261D874E38E048F05FF12614B
:1033DD00C88D48800375480090006EE0600575BB90
:0633ED001A800375BB18F5
:10359F00022C83022E3D022FDE0230930230F802FE
:0B35AF0031A102323E0232750233A34C
:0533F300054CD2EC22A4
:09620A002582F582500205832271
:0F008C0025E050020583258250020583F582226C
:1061A700EF2F500205832582F582E5833E2EF58386
:0161B70022C5
:10621C00CFC39FFF50011E22C3EF9DFFEE9CFE22B9
:08622C000806B6000218062264
:0D61E600A3E004F07006120049E004F0226E
:0E003900048007C3CE13CECF13CFD5E0F6223E
:1060C600BC000FBE0008ED8FF084FFADF022E4FEA9
:1060D600FF22BE000DEF60FE54F0606F20E7030262
:1060E600617CEAC0E0EBC0E078017A0075F001EE71
:1060F60020E710EF25E0FFEE33FE0AC5F023C5F0DA
:1061060030E7F0EA5407F9096A7A007B0060010873
:10611600C3EC9E40167004ED9F4010ED9FFDEC9E73
:10612600FCE5F0CA4ACA03F5F08005E5F003F5F090
:10613600C3EE13FEEF13FFD9D77908CACBCAD8D05E
:10614600EAFEEBFFD0E0FBD0E0FA22EC8FF084FC15
:10615600ED54F045F0C48FF084FEEDC454F045F0E4
:10616600C48FF084FDEEC4FE54F02DFFEE540F3CB8
:10617600FEADF07C0022790078008FF0EC7E0820DE
:10618600E70DC3CD33CD33C933C9C833C8DEF08478
:1061960049F9E5F08FF0BE00E6FD7C00E9FFE8FE78
:0161A60022D6
:0E61D800F88FF0A4FFE5F0CE88F0A42EFE2292
:10000300EF8DF0A4F9A8F0EF8CF0A428F8EE8DF0B2
:06001300A428FEE9FF2213
:1061B800600D782B0261C2007830D8FED5E0F82255
:1061C800EEC0E07E001260C6EFFDEEFCD0E0FE22DD
:0C61F300EEC0E07E001260C6D0E0FE228C
:03001B0002001EC2
:0300530002005652
:03009B00020071EF
:0300000002621386
:0962130075817C75D0000243681E
:0B61FF00E5822FF582E5833EF5832248
:0A0049000582D5820215831582227C
:10001E00C0E0C0F0C083C082C0D075D00012430FC4
:0B002E00D0D0D082D083D0F0D0E032E0
:10005600C0E0C0F0C083C082C0D075D00012431289
:10006600D0D0D082D083D0F0D0E032C0E0C0F0C093
:1000760083C082C0D075D000124331D0D0D082D098
:0600860083D0F0D0E0324F
:00000001FF
